:040000008A018E28BB
:08000800F100F10E030EF200FD
:10001000040EF3000A0EF4008A01831203130C0885
:100020002039FF39003C03191C288C208A110A1240
:100030000B11831203138C120B080239FF39003C99
:1000400003193C2800008B1080307502031D2F28F7
:10005000C030831603138100C030F500352880308E
:100060008316031381008030F5003B3083120313A5
:1000700081000B118B1681280B080439FF39003CD5
:10008000031981280B118B12030183120313081823
:100090000130FD0007307602031CF90A01307D02B1
:1000A00003195928F6013130FB008D208A110A12FC
:1000B00080280630760203186428F60A3030FB00E8
:1000C0008D208A110A12802806307602031D8028AE
:1000D00079080139FE00FE08031D7B28F60A0D3061
:1000E000FB008D208A110A120A30FB008D208A1134
:1000F0000A12F90180283030FB008D208A110A1283
:100100000B11740E8A00730E8400720E8300710E40
:100110000900C428EF2801290E292629F801F70132
:100120000730F600F90189208A110A12FC012A30F1
:10013000FA008B208A110A120D30FA008B208A11E6
:100140000A120A30FA008B208A110A127808031961
:10015000A6287C08FC0A203E840083130008FA00CD
:100160008B208A110A1214307C020130031803011B
:10017000FF390130031D0030003C031DFC017808ED
:10018000031DF803A628A6288B018030F5008030D7
:1001900083160313810083129F01063083169F008C
:1001A0000130850083128501F130831686008312A9
:1001B00086019930831687008312870101308316E8
:1001C0008800831288010130831689008312890117
:1001D0008C018A208A110A12D0308B000800831209
:1001E000031398171813831618131930990018154C
:1001F000181298168C16831218168C120B178B1760
:1002000008008316031318080239003C031D09294E
:1002100001297A088312031399000800831203133B
:1002200018080639003C031D1E291A08FB008D2002
:100230008A110A1283120313181622298312031338
:1002400018121816831203131A08080014307702C4
:10025000013003180301FF390130031D0030003C59
:10026000031DF7017B08F0007708F70A203E8400A1
:100270007008831380007808143C0130031D0301CB
:10028000FF390130031D0030003C031DF80A08004F
:00000001FF
